:10000000000000000000882AA500841780048413E3
:10001000FA30B200B301C621A60AAF0AAA01AB01A9
:1000200000082505B200000000082505B3003206CF
:10003000330525060319AA0A0319AB0A3308B200CF
:10004000AE030319AF030319A60B13282A08DC29F2
:100050008030A100FE305421013054217530A700BA
:1000600030306529A101A117B600B608031D3A2852
:1000700003013B280130B6020310A20CA20CA20C13
:10008000C0302205403EB607FE30542136085429C0
:10009000A101A117B600FE30542136085429A01141
:1000A00024080319A0150530A3002730AB00103039
:1000B00065200330AB00E8306520AB01643065207B
:1000C000AB010A3065202E086C28AA002F08A70073
:1000D0002E08A600AA212608A600A3030319A01132
:1000E000240803197628230203187D282608031DF7
:1000F000A011A0197D28303E54290800C900BA1F5C
:1001000083282D305421BC0F8A28BB0F8A28BA0AB5
:100110000319BA0AC101C201C301C401BA176A3086
:10012000B9070310BA0CBB0CBC0CC40CC30CC20C3A
:10013000C10CB90F91283C083902BC07B9023B0831
:100140003A02BB07BA02A401DD202E305421CA01B5
:100150000310410DBC00420DBB00430DBA00440D1D
:10016000B900CA0D0310BC0DBB0DBA0DB90DCA0DF7
:100170004108BC0742080318420FBB074308031895
:10018000430FBA0744080318440FB9070318CA0FEE
:100190000310BC0DBB0DBA0DB90DCA0D4A08303E97
:1001A00054213C08C1003B08C2003A08C30039088A
:1001B000C400C90BA7280310DC29A0112408031DC3
:1001C000E428A0150A30A4003C08A9003B08A800B8
:1001D0003A08A7003908A600A301B101B001AF0198
:1001E0000A30AE007421A30A23082402031DED285F
:1001F0002E08031DA011A01DFF28240B02292E0884
:10020000303E5421A40BE428DC29B30006118611EA
:100210008316061186110F30860583123308A01845
:100220002F293E30A700803065213330B2004321B2
:100230001330A700883065214321643064214321B5
:10024000643064212230B200432128302E210C304A
:100250002E2106302E21A01433082F292014B2009D
:10026000201C3D298611033C031C422942210730F2
:10027000A700D0306521031408002014FE3C0319A8
:1002800052298615201C201006150F3086053208CD
:10029000F039860400000611B20E00002018432930
:1002A000323064213308DC29A11B05290800AB0189
:1002B000AA00FF30AA07031CAB07031CDC2903308C
:1002C000A700E63065215929A701FC3EA600A70931
:1002D000031C7029FF300000A60703186B29A6072E
:1002E0000000A70F6A290800BD01BE01BF01C001BF
:1002F0002130AC009B29BD0DBE0DBF0DC00D2E08D9
:100300003D022F08031C2F0F3E023008031C300F44
:100310003F023108031C310F4002031C9B29C0001F
:100320002E08BD022F08031C2F0FBE023008031C2D
:10033000300FBF020314A60DA70DA80DA90DAC0B1D
:100340007B294008B1003F08B0003E08AF003D08DF
:10035000AE00DC29AF01AE011030B200270DAE0DAA
:10036000AF0D2A08AE022B08031C2B0FAF02031897
:10037000C0292A08AE072B0803182B0FAF0703105C
:10038000A60DA70DB20BAE29260808001030B80044
:10039000A701A601B30CB20C031CD4292A08A60796
:1003A0002B0803182B0FA707A70CA60CAF0CAE0C3D
:1003B000B80BCA292E080800831383120313080000
:1003C0004208BF004606CC004108003A031D45081C
:1003D000003A0319302AC1077E30031CF329C102F9
:1003E0000318322AF629C102031C2F2A4408BD0033
:1003F0004308BE00BF17C617C401C301C2011830AD
:10040000CD00BF0CBE0CBD0C031C102A4808C4074D
:1004100047080318470FC30746080318460FC207CB
:10042000C20CC30CC40CCD0B012AC21B1F2AC40D65
:10043000C30DC20DC10803192F2AC1033F0D031CB0
:100440002E2AC40F2E2AC30F2E2AC20F2E2A0314BF
:10045000C20CC30CC40CC10A0319322A392A4B1529
:10046000C101352ACB14FF30C100C401C301803063
:10047000C200CC1B3C2AC213DC29C301C401CC132B
:10048000502ACC13C41F502AC409C309C209C10988
:10049000C10F4F2AC20F4F2AC30A0319C40ACC172F
:1004A0009630CD00C40803195E2A0830CD074208F3
:1004B000C1004308C2004408C300732AC308031DD7
:1004C000732A0830CD024208031D6F2A0830CD027E
:1004D0004108031D6E2A4408CD007D2AC101C300D6
:1004E0004108C200C101C31B7B2A0310C10DC20D0C
:1004F000C30DCD03732ACC1FC3134108C4004D089C
:10050000C1004308CD004208C3004D08C200DC29E9
:10051000831203134030CB00A00107309F004F30FF
:100520008316850003308600073083129F00FE305B
:100530000521403005210E300521113005211030F4
:1005400005211030052110300521153005210E3010
:10055000052100300521FE300521483005210A30F3
:1005600005210E30052111300521113005211130F2
:100570000521113005210E30052100300521FE3006
:100580000521503005210A30052111300521113097
:1005900005211130052111300521113005210E30C2
:1005A000052100300521FE30052158300521043099
:1005B00005210E30052104300521043005210430C9
:1005C0000521043005210E30052100300521FE30C3
:1005D0000521603005210E30052111300521103034
:1005E00005210E30052101300521153005210E3081
:1005F000052100300521FE300521683005210E302F
:100600000521003005210F3005211030052117305C
:100610000521113005210F30052100300521FE3064
:100620000521003005210030052100300521093069
:10063000052109300521093005210E30052108303A
:100640000521643057212820CF01CE01D101D001EE
:10065000D501D401D301D201D901D801D701D601E6
:10066000DA01DC01DE01DD01DB01D9240730AB005A
:10067000D030582128208030A100C030482043309D
:1006800005215030052153300521C6304820433024
:100690000521503005214D300521CA304820073052
:1006A000052153300521763005212F300521683092
:1006B00005210330AB00E830AA0005308400023089
:1006C0000420CE002B08CF0003304F02031C6E2BFA
:1006D000031D4B2CE8304E0203184B2C8030831244
:1006E0000313A100CF3048202A300521CF08031D75
:1006F0008A2B0A304E0203188A2B8030A100482032
:10070000203005210521A4014E08AE004F08AF009E
:100710004F20A62BCF08031D9D2B64304E020318DB
:100720009D2B8030A100482020300521A4014E08D7
:10073000AE004F08AF004F20A62B8030A10048200C
:10074000A4014E08AE004F08AF004F20DC0A4E084F
:10075000D0074F080318013ED1073C305C02031D4F
:10076000B22BBB23323057218030A100CF3048203C
:10077000203005213B2BD108031DD22B093050021C
:100780000318D22B8030A10084304820203005216E
:10079000052105210521A4015008AE005108AF0034
:1007A0004F201B2CD108031DE82B63305002031887
:1007B000E82B8030A100843048202030052105211D
:1007C0000521A4015008AE005108AF004F201B2C9A
:1007D00003305102E730031950020318FD2B80301B
:1007E000A10084304820203005210521A4015008B3
:1007F000AE005108AF004F201B2C273051020F30A4
:10080000031950020318112C8030A10084304820B5
:1008100020300521A4015008AE005108AF004F2040
:100820001B2C8030A10084304820A4015008AE0069
:100830005108AF004F205008C1005108C2003D22AE
:100840001130C800C730C7003A30C6007730C50045
:10085000E0214408D5004308D4004208D3004108F1
:10086000D2008030A1008A3048205508BC005408CE
:10087000BB005308BA005208B90002307E20DC01E8
:10088000D101D001D501D401D301D201CF01CE01D4
:1008900032305721080028208030A10085304820C0
:1008A00059300521023005214B30052153300521F7
:1008B000453005214B30052120300521052105213A
:1008C000052105218030A100C1304820523005218A
:1008D00041300521443005215930052141300521A1
:1008E00053300521593005214F3005214E30052167
:1008F0002030052121300521052105212030052149
:1009000005210330AB00E9305821282003304F0285
:10091000031CD72C031D902CE8304E02031CD72C4F
:10092000033083120313AB00E830AA0005308400C3
:1009300002300420CE002B08CF008030A1004820D8
:100940004330052150300521533005213A3005212F
:10095000A4014E08AE004F08AF004F208030A10028
:10096000C03048200730052153300521763005215D
:100970002F300521683005213A3005214E08C1008D
:100980004F08C2003D22A030C8001A30C7002F30E7
:10099000C6007D30C500E0214408BC004308BB0010
:1009A0004208BA004108B90002307E20862C282077
:1009B0003B2B1030DB0002305B02031CF52C803037
:1009C000A1000130A2005B0834202A3005218030CC
:1009D000A1000130A2005B0A3420203005212D3017
:1009E00057210130DB020318DB2C1030DB00043010
:1009F0005B02031C112D8030A1000130A2005B08B6
:100A00003420543005218030A1000130A2005B0A5F
:100A10003420203005212D3057210130DB0203180E
:100A2000F72C1030DB0006305B02031C2D2D8030CC
:100A3000A1000130A2005B08342041300521803044
:100A4000A1000130A2005B0A3420203005212D30A6
:100A500057210130DB020318132D1030DB00083062
:100A60005B02031C492D8030A1000130A2005B080D
:100A70003420323005218030A1000130A2005B0A11
:100A80003420203005212D3057210130DB0203189E
:100A90002F2D1030DB000A305B02031C652D8030E7
:100AA000A1000130A2005B083420453005218030D0
:100AB000A1000130A2005B0A3420203005212D3036
:100AC00057210130DB0203184B2D1030DB000C30B6
:100AD0005B02031C812D8030A1000130A2005B0865
:100AE0003420493005218030A1000130A2005B0A8A
:100AF0003420203005212D3057210130DB0203182E
:100B0000672D1030DB000E305B02031C9D2D803002
:100B1000A1000130A2005B0834202A30052180307A
:100B2000A1000130A2005B0A3420203005212D30C5
:100B300057210130DB020318832D8030A1008E3055
:100B400048202030052105210330AB0020305821FA
:100B50008030A100C03048205230052141300521AD
:100B600044300521593005214130052153300521FC
:100B7000593005214F3005214E3005212030052107
:100B8000013005214C3005210030052102300521BE
:100B900043300521023005210730AB00D030582109
:040BA0000800D12D4B
:02400E00223F4F
:00000001FF
